:03000000021C449B
:0C1C440078FFE4F6D8FD7581DD02003663
:0100190022C4
:061913008B2D8A2E892FA6
:10191900750A027F48121A75121C80EF20E0F9AB94
:101929002DAA2EA92F120973787FE6FE08E6FDED90
:01193900FFAE
:01193A00228A
:100F3300434647002D53322D0052415445434C52F2
:100F430020554E49544C49544554524947545245EF
:100F5300565354525453544F505A45524F4241558D
:100F63004444464C54534156455253542050432015
:100F7300205F3120735F3220735F3520733120731C
:100F830020322073203520732031302073333020FA
:100F93007331206D2032206D2035206D20313020BB
:100FA3006D3330206D312068200000000100020005
:100FB30005000A001400320064012C025804B00B2F
:100FC300B8177046508CA0010204081030466565BE
:100FD30074596172644D6574724F6666204F6E205A
:100FE300204E6F2020596573204F66662054696D2B
:100FF30065416C7420547269674F66662054726948
:0910030067537472745265632096
:1019D50025E024ACF582E4340FF58322052FE52FAD
:1019E500C3940222A62FE52F75F004A42208F60859
:0419F500F608F622D8
:10161400789F76AB0876CD08760008760AE408F65B
:1016240008760108F60876640876401219F208F67E
:1016340078ADF608760A08F608763C08F6087614BB
:0F16440008F608760F1219F278BA76050218C068
:10180800750E1D750FC012143978A0E664CD7004EA
:1018180018E664AB600312161478B9E6FFF46003A7
:0F182800EF700478B9760478BAE6B4FF0276055B
:01183700228E
:101B0A00C2AF5387DF7DC07C1DE4FF121B324387BF
:031B1A0020D2AF27
:011B1D0022A5
:10143900753AFF850E3B850F3C753D00753E00757D
:101449003F9FE4FFAB3AAA3BA93C8F827583001208
:101459000946AB3DAA3EA93F8F82758300120985D3
:101469000FBF1CE078B8E6FFF46003EF700478B8AA
:0A147900760478B9E6B401027604A7
:011483002246
:1018C0007D01E4FF121A3A121B0AC2AF5387DF7F71
:1018D0009F7B1C7DC07C1D121B3C438720D2AF7FA9
:0A18E00002121737E4FDFF021A3A66
:10047B00E4F52D7BFF7A0F79331215D47F05121714
:10048B0037A297829650FAA2969218A2979219E5E4
:10049B002D75F004A4243CF9740F35F0FA7BFF1290
:1004AB0015D47F05121737852D2EE4F52F7BFF7A98
:1004BB000F79371215D4E52DB40A00400302054914
:1004CB009004D2F82828730204F0020549020511A2
:1004DB0002051902051D02052502052D0205310233
:1004EB0005390205417F01EF1219D578A1E6FC0809
:1004FB00E6FD7401936D7003E4936C70028F2F0F04
:10050B00BF0FE40205CF78A3E6F52F0205F278A41E
:10051B00800278ACE6F52F02060C78ABE6F52F02DD
:10052B00063A78B5800278B6E6F52F02065778B70B
:10053B00E6F52F02068C78BAE6F52F0206B2E52D0A
:10054B00652E600302049AA218309601B35013A2D1
:10055B0096921830960C052DE52DC3940D4003E4AF
:10056B00F52DA219309701B350D4A2979219309759
:10057B00CDE52DB40D0050C690058AF828287302DE
:10058B0005B10205DA0205E00205FE0206180206B5
:10059B002C02064502066202067A0206A00206C378
:1005AB000206C90206CF052FE52FC3940F40037532
:1005BB002F01E52F1219D5E493FF74019378A1CF86
:1005CB00F608EFF61219EB2470F9740F0206951268
:1005DB0012F0020549052FE52FC394034003E4F500
:1005EB002F78A3A62FE52F75F004A424D0F9740F50
:1005FB000206951219E14003E4F52F78A4A62FE526
:10060B002F75F004A424DCF9740F0206951219E17E
:10061B004003E4F52F78AC1219E924DCF9740F8050
:10062B00691219E14003E4F52F78ABA62FE52F757E
:10063B00F004A424E4F9740F8050052FE52FC39424
:10064B00044003E4F52F78B5A62FE52F75F004A42D
:10065B0024ECF9740F8033052FE52FC3940340036B
:10066B00E4F52F78B61219E924ECF9740F801B0509
:10067B002FE52FC394044003E4F52F78B7A62FE59D
:10068B002F75F004A424FCF9740F35F0FA7BFF12DC
:10069B0015D4020549052FE52FC394064003E4F555
:1006AB002F78BAA62FE52F900FCA9375F018A4FFD9
:1006BB00AEF012121F020549121614020549121848
:0A06CB00C002054943A208020549D8
:0A1C5C004552415300444F4E45002D
:101BBC0078A1E6F55408E6F55522E573AE72780681
:011BCC0022F6
:10109F00C216C21778B9E6FFE4FCFDFEFB7A20F911
:1010AF00F81209A78F798E788D778C76E47B40FACA
:1010BF00F9F8120A328E708F71E4F52EF52FC3E511
:1010CF002F9571E52E9570501CE52D64816016AF3C
:1010DF002FAE2E121838121B1E8F2D052FE52F70D5
:1010EF00DD052E80D9E52DB48108E52F152F70026F
:1010FF00152EE52F65717004E52E6570700CD216F4
:10110F00121C0EE4F572F5738007852E72852F730E
:0B111F00E4F574F575755380121BBCDD
:01112A0022A2
:10183800C3EF9571EE95705024EF7806C333CE331D
:10184800CED8F9FD750A02EE787FF6CFEDCFEF0816
:0D185800F67F50121ADE121C80EF20E0F91E
:011865002260
:031AAB00CDEFCDAF
:101AAE00750A02EE787FF6ED08F67F50121ADE12F6
:061ABE001C80EF20E0F99E
:011AC40022FF
:101B1E00750A017F50121A75121C80EF20E0F978B9
:031B2E007FE6FF50
:011B31002291
:101AF500121AABE4FFFE0FBF00010EBE0FF8BFA028
:041B0500F5121B1E9C
:011B090022B9
:06176D00CBEFCBCAEECA6F
:10177300301603301727750A03EA787FF6EB08F66D
:1017830008EDF67F50121ADE121C80EF20E0F9E418
:0D179300FFFE0FBF00010EBE0FF8BFA0F556
:0117A0002226
:10155200753000753100753253E4F52F121BC6C386
:1015620033CE33CED8F97C00252FFFEC3EFEAB30D4
:10157200AA31A932852F82758300120946FD1217FE
:101582006D052FE52FC3940640D27574007575065C
:011592002236
:1011A7008E2D8F2E121BC6C333CE33CED8F925759D
:1011B700FFE5743EFEEEC0E0EFC0E0E52DFDD0E0B8
:1011C700FFD0E0FE12176D0575E575700205741204
:1011D7001BC6C333CE33CED8F92575FFE5743EFE63
:1011E700AD2E12176D0575E575700205740557E587
:1011F7005770020556C3E5759440E574940040178F
:10120700E4F574F5750573E573700205729571E57C
:081217007295704002D216220C
:1012F000E4F574F5757BFF7A1C795C1215D4D2176E
:10130000E4F53AF53BC3E53B9571E53A957050211C
:10131000E53BAE3A7806C333CE33CED8F9F5758EB9
:10132000747D81FF12176D053BE53B70D8053A804F
:10133000D4C2177BFF7A1C79611215D4E4F572F5DB
:0713400073F574F575C21688
:011347002283
:10129700E4F53AF53BF53CF53DC3E53D9571E53C95
:1012A70095705044E53B6481603EAF3DAE3C1218FB
:1012B70038121B1E8F3BE53B64807022AF3A053A1C
:1012C700FCFDFEFBFAF9120B337F2C120016AE3C25
:1012D700AF3DE4FCFDFBFAF9120B33121C70053D20
:0812E700E53D70B5053C80B146
:0112EF0022DC
:021484008F3A9D
:10148600E4F53BF53CF53DF53EC3E53E9571E53D9E
:1014960095705030E53C6481602AAF3EAE3D12182F
:1014A60038121B1E8F3CE53CB4800FE53B653A7055
:1014B60007AF3EAE3D021838053B053EE53E70C916
:0414C600053D80C59B
:0114CA0022FF
:10159300121BBC78ACE6F558E4F556F55712155214
:1015A30085727A85737B7F0112198930021A78AFAD
:1015B300E6FE08E6FFE4FCFD7B64FAF9F81209A7EE
:1015C3008F6F8E6E8D6D8C6C300505C205121C37C6
:0115D30022F5
:10168E0085722D85732EE57545746008052EE52E41
:10169E007002052D857A72857B73121552852D7217
:1016AE00852E73C3E52E9571E52D95704007E4F5F3
:0A16BE0072F573D2167F020219893B
:101B3200740478FF769612FF0322740078FF76967B
:041B420012FF032269
:03003300020D6457
:100D6400C0E0C0F0C083C082C0D0E8C0E0E9C0E009
:100D7400EAC0E0EBC0E0ECC0E0EDC0E0EEC0E0EFC4
:020D8400C0E0CD
:100D8600E5D954F8FF120B0D0DB3080DB3100DC2C3
:100D9600180DDD200DC4280DDD300DDF380DE540C2
:100DA6000DDD480DFE500E1B5800000E29850DDA8C
:100DB600C2DDC2DC750B00750C008070800EE50A82
:100DC60070028056050CE50C7002050B1200268F8A
:100DD600DAC2DDC2DC80558016D2DDC2DC804DC2AF
:100DE600DDC2DCE50A7004C2DA8041D2DA803DC297
:100DF600DDD2DC7508048034AFDA121C50050CE530
:100E06000C7002050BC2DDC2DCE50A7004C2DA8092
:100E16001BD2DA8017AFDA121C50C2DDD2DC75089D
:0E0E2600028009750804C2DDC2DCD2DAC2DB2C
:100E3400D0E0FFD0E0FED0E0FDD0E0FCD0E0FBD07D
:100E4400E0FAD0E0F9D0E0F8D0D0D082D083D0F06E
:030E5400D0E032B9
:1018940043910C43920CE4F5DBEF25E0F5DB3018C3
:1018A4000343DB0175DD1775DC1775D84453F8FE67
:0C18B40053F7FE43F701E4F508D2E822E8
:101ADE00E50830E002FF22E4F509750803EF25E082
:071AEE00F50DD2DD7F02229D
:101A7500E50830E002FF22E4F509150A750805EFCF
:0B1A850025E04401F50DD2DD7F0222B8
:061C800020DBFDAF08228D
:0D002600150AAF090509747F2FF8E6FF22C7
:0C1C5000747F2509F8EFF60509150A223B
:0D1C2A007584C075853F53913F759200226F
:101962006F035D5733767E437F771004007B3E6CB6
:101972001F7C78773B020F382C5A1A6F79751876CC
:071982003C0E2F4E2B375DD8
:1017D5004EFECCEFCC0F747F2CF8EEF6EDC4332221
:1017E50090196EE493FF78D3F608EFF608F608F63D
:1017F50022E493FF74D32EF8EFF60E22EE3395E034
:03180500FDFC22C5
:10100C00E4FF0F247FF876CD0F747F2401F87680EF
:10101C000F747F2402F876E00F747F2403F876F8BF
:10102C00301A0A0F747F2404F87671800ACEEFCE42
:10103C000F747F2EF8767078D3E6FEC4540FFDCC77
:10104C00EFCC0F747F2CF8EDF6EEC454F0FE78D490
:10105C00E6FD131313541F1217D554E0FE78D5E692
:10106C00FD1313543F1217D53354C0FE78D6E6FD4A
:10107C00C3131217D533335480FECDEFCD0F747FCD
:10108C002DF8EEF68F0A7F38121ADE121C80EF2034
:02109C00E0F979
:01109E00222F
:1017A100C21A1217E5750A0A787F76CD0876800885
:1017B10076E00876F80876700876050876D508761A
:1017C1009B0876FFE408F67F38121ADE121C80EFC0
:0317D10020E0F91C
:0117D40022F2
:101A9000EF24F9600B14600C2402700EC21A800748
:0B1AA000D21A80031217E512100C226E
:10134800C3EF648094E1400ED3EF648094FA5006B2
:10135800EF24ACFF803CC3EF648094C1400ED3EF10
:10136800648094DA5006EF24CCFF8026C3EF6480B3
:1013780094B0400ED3EF648094B9500674D02FFF18
:101388008010BF2D047F0A8009BF5F047F0B800295
:031398007F0C22A5
:10193B00CEEDCECDEFCDCFEECF121348EF3395E0FA
:10194B00FE74622FF58274193EF583E493FF74D312
:07195B002DF8EFF602100C5D
:0615D4008B3C8A3D893EBC
:1015DA00E4FE90196E1217F6BE04F7E4FEAB3CAABD
:1015EA003DA93E8E82758300120946FF60191213C7
:1015FA0048EFFD3395E0FC74622DF58274193CF5D1
:0A160A00831217F6BE04D602100C7E
:04121F008F828E83A9
:101223001218017B197AFC79FF78FFD3120AD24096
:101233000390FC19AF82AE83121801E47B0F7A2767
:10124300F9F8C3120AD2500390270FE4F53074CE95
:101253002530F8E4F60530E530B405F2AE83AF820D
:101263001218017B007A0079CE120B3378D1E67025
:101273001A75300374CD2530F8E6FF74CE2530F8A7
:10128300EFF6D530EF78CE762080E17B007A0079D7
:04129300CE0215D49E
:101B9600C213C215C212E4FDFF121A3AE4FD7F0118
:031BA600021A3AE6
:101A3A00EF146011047016BD0104C2828002D282C2
:0E1A4A00A282921422BD0103C28122D2812207
:10198900EF24FE600D14601124027019D213757DC5
:101999000122C213A214928222D215757E027D0100
:0619A9007F01121A3A2230
:1018EA00301312D57D0F308207C282757D0F8005B5
:1018FA00D282757D23E57ED39400400CD57E09C241
:09190A0015E4FD7F01121A3A22D6
:101B460046554C4C005A4C4F470020342D32005419
:041B56007269670049
:10186600F564F563F562F561856052855F51855EC5
:1018760050855D4F22E6FE08E6FFE4FCFDAB60AA5C
:0E1886005FA95EA85D2278D7E6FE08E6FF2285
:030013000219F9D6
:1019F900C0E0C0D075D010200E0CAF8DEFAD8BF5C7
:101A090069EDF56AD20E758D00758B00D0D0D0E0E6
:011A1900329A
:021737008F3BE6
:10173900E4F53CF53DC3E53D953BE53C940050237C
:10174900900000AF82AE83E4FCFD7B207A4EF9F86D
:10175900D3120AD24003A380EA053DE53D70D605C0
:031769003C80D2EF
:01176C00225A
:0E1C0E007BFF7A1B79461215D47F0A02173726
:0F1BFF00D20C301606121C0EC20C2212159322A5
:05000E00C20C02168E79
:0D1C3700E4121866F560F55FF55EF55D22BC
:101BEF008E2D8F2EEEFF120016AF2EE52E02001651
:10003600121C2A121C66121B967F04121737209771
:100046000B7D057F0112112BD2AF80FE209612D2B6
:10005600AF121808C2187F7012189412109F12045B
:100066007B12180878BAE6FDE4FF12112B438720AD
:10007600D2AFC2187F701218947F01121737121070
:100086009F1217A17A1B794B1204707A1B795012B2
:100096000470120019E478DDF61216537F01121768
:1000A6003712001AA2969208A2979209E4F524F54F
:1000B6005CF55BF55AF559F5257564F17563D875E8
:1000C60062FF7561FFF552F551F550F54FC20AF51D
:1000D60060F55FF55EF55DC20DC211C20CF526F541
:1000E60027F569F56AC20EF56BF568F567F566F5ED
:1000F60065F56FF56EF56DF56CC20FF52078A4E623
:100106006004D2808002C28078B5E624FE600B14BB
:10011600600C2402700AD2018006D2068002D20048
:1001260078B6E624FE6007047006D2028002D20783
:1001360078B7E624FE600B14600C2402700AD20322
:100146008006D2048002D20530011CC20178ADE6D9
:10015600FE08E6FFE4FCFD7B64FAF9F81209A78FB6
:10016600688E678D668C6578DDE6C3940240F8E498
:10017600F6209605209702D21030963030972D3013
:10018600102AC210AF52AE51AD50AC4FEC4D4E4F8F
:1001960070051218668011E4F564F563F562F56181
:1001A600F552F551F550F54FD209D208A20830960E
:1001B60001B3501CA2969208309615201012C20167
:1001C600300A06C20A7F068004D20A7F07121A90F6
:1001D600A209309701B35017A297920930971020C1
:1001E600100DB20C300C05121BFF800312000E120C
:1001F60006D5AF68AE67AD66AC65EC4D4E4F602672
:1002060074FF2FF568EE34FFF567ED34FFF566EC05
:1002160034FFF565AF68AE67AD66FC4D4E4F7006B0
:10022600200C03121BFFAF6FAE6EAD6DAC6CEC4DC8
:100236004E4F602374FF2FF56FEE34FFF56EED34ED
:10024600FFF56DEC34FFF56CAF6FAE6EAD6DFC4D2A
:100256004E4F700312000E200E03020305C2AFC2FA
:100266000ED2AFE4856A2C85692BF52AF529AF2CC9
:10027600AE2BAD2AAC297B107A27F9F81209A78F85
:100286002C8E2B8D2A8C29E4FB7A90F9F81214CB4C
:100296008F2C8E2B8D2A8C2978ABE66009C374B817
:1002A6009FFF740B9EFEE56B14601624FE602024EF
:1002B600037049C3EF94B0EE9404500E756B018041
:1002C60009D3EF9414EE94054035756B038030C363
:1002D600EF94B0EE94045027756B01300006200CA5
:1002E60003121BFF300305C203121C37300C02D267
:1002F6000F7BFF7A1B79551215D48003E4F56B0545
:1003060025E525C39401500302046AE4F525FB7A2A
:1003160000792812191378D7EEF608EFF6E5286467
:1003260002600302046A12188C78A3E6FD1213ED2C
:10033600E55C2FF55CE55B3EF55BE55A3DF55AE578
:10034600593CF5590524E524C39405500302046A73
:10035600AF5CAE5BAD5AAC59E47B05FAF9F8121402
:10036600CB8F5C8E5B8D5A8C59C3E55C9552F55CE0
:10037600E55B9551F55BE55A9550F55AE559954F6C
:10038600F559AF64AE63AD62AC61AB5CAA5BA95ACA
:10039600F8D3120AD2400C855C64855B63855A6289
:1003A600855961300A0AAF6478D9E563F608EFF635
:1003B600AF5C78D7E55BF608EFF6300A03088002F3
:1003C60078D7E6FE08E6FF12121F30110612188CC7
:1003D600121BEF0527E52770020526C378A296E5CE
:1003E6002618964038E4F526F527300D0612188CA7
:1003F600121BEF300C277F0312198920161978ACCF
:10040600E6600C300F097F007E821211A7C20F1220
:10041600188C1211A78006121C0E12000E855C6045
:10042600855B5F855A5E85595DE4F55CF55BF55A3B
:10043600F559F524300405C204121C37300611782C
:10044600B112187BD3120AD24006200C03121BFFEE
:1004560030071178B312187BC3120AD25006300C3B
:0A0466000312000E1218EA02016DE5
:0B0470007BFF1215D47F041217372207
:1019AF00444C0021536967005A4C4F47004D4F4438
:1019BF0000342D32004A756E2032332032303037EA
:0619CF000050524F4700DA
:10150F00AF35AE34AD33AC32EC4D4E4F22EF24FF3E
:10151F00F535EE34FFF534ED34FFF533EC34FFF5EC
:10152F003222E475352075344EF533F53222E475E9
:10153F003501F534F533F53222752F00753000750E
:03154F00319F22A7
:1006D500121C1CEF700302090D121A58EF120B0DB4
:1006E50008D42408DF2A08F84808CC4D08E4500847
:1006F500245207166107A66309026807F96C07FF0C
:100705007207FC73082874089C760897780000091E
:100715000DC20A7BFF7A1979AF1215D41215311261
:100725001C1CEF700A12150F600512151C80F012C3
:10073500150F700302090D121A588F2E121484E436
:10074500F535121541E47F06FEFDFCAB35AA34A94B
:1007550033A832C3120AE8501F121B1E8F2E120037
:1007650016E5352401F535E43534F534E43533F54E
:1007750033E43532F53280CD121B1E8F2EE52E6403
:10078500806016E52E64816010120016121B1E8F04
:100795002E120016752D018003E4F52DE52D70D878
:1007A5002212154812153DF52E12150F602412154B
:1007B50031121C1CEF700A12150F600512151C80F2
:1007C500F012150F600312090E052EE52EC3941CB9
:1007D50040D712150F601A789FB6AB0708B6CD0340
:1007E5000208DC7BFF7A1979B21215D47F0A021749
:1007F50037020894B20D22021297121548E4F52E1D
:10080500AB2F0531E531AA307002053014F9120914
:100815002DFF120016052EE52EC3941C40E222433F
:10082500A20822C20A752F007530007531DB12153A
:100835003DF52E12150F6024121531121C1CEF7098
:100845000A12150F600512151C80F012150F6003B2
:1008550012090E052EE52EC3940240D712150F601E
:100865002E78DBE6FE08E6FFEE3395E0FDFCC3EFF0
:100875009560F539EE955FF538ED955EF537EC95B4
:100885005DF536AF3978A9E538F608EFF680480208
:100895001439C20A0212F07A1979B71209227A19A3
:1008A50079BC121BA978B8E62430FF120016121C79
:1008B500707F761200167A1979C01209227A197991
:1008C500C4121BA9021C70E4F52EAF2E020016C23D
:1008D5000AE478A9F608F60218C0C20A021614C27C
:1008E5000A7BFF7A1979D01215D47D017F01121187
:1008F5002B80FE7D03E4FF12112BD2112278BAE67C
:08090500FDE4FF12112BC211E9
:10090D0022121A58AB2FAA30A931852E8275830079
:10091D00EF120985227BFF121BA9121C707BFF228F
:0A1C6600E4F5955396BF53A27F22C8
:101653005389F0438901538FFE758C70E4F58A53E7
:10166300B8FD53B7FDD2A9D28C53890F4389905348
:101673008FEFF58DF58B4391105392EF53B8F753DA
:0B168300B7F7D2ABD28ED28AD2AA22D7
:03000B00021BCD08
:101BCD00C0D075D01878DD06758C70758A00D0D0B0
:011BDD0032D5
:03001B00021C794B
:071C7900758D00758B003230
:101B5A000D0A003031323334353637383941424391
:041B6A0044454600A8
:101B6E00AF4EAB42AA43A944054E22AF41AE40ADA3
:041B7E003FAC3E2218
:10112B005387BF75985053877FE4F5BABF010543CA
:10113B00A240800353A2BFE4F5BDED14601514600B
:10114B001A14601F1460242404702575BEF075BF3B
:10115B000B802375BEF075BF05801B75BEF075BF88
:10116B0002801375BE7075BF01800B75BEB0800316
:10117B0075BE30E4F5BF75BD035391FE4392014339
:10118B0091025392FDC21B53B8EF53B7EF43B81004
:0C119B00E478CCF618F678CDF6D2AC2241
:03002300021700C1
:10170000C0E0C0D0E8C0E030981E78CCE6C3940FAB
:10171000501418E60624BBF8A69978CC0618E6C340
:10172000941040027600C298309904C299C21BD02E
:07173000E0F8D0D0D0E03258
:08000300201BFDD21B8F992286
:101A1A0078CCE6D39400401508E60624BBF8E6FF26
:0F1A2A0078CC1608E6C394104005E4F6227F003E
:011A3900228A
:03001600020003E2
:101A58007F207E4E78CCE67010D3EF9400EE940091
:0C1A68004007EF1F70EE1E80EB121A1AF0
:011A7400224F
:101BA90012092DFF600C120016740129F9E43AFAA2
:031BB90080EE2299
:0E1C1C0078CCE6D3940040037F01227F0022A3
:101AC500CEEFCEEE54F0C4540F901B5D93FF120081
:091AD50016EE540F93FF020016F7
:101BDE00CDEFCDCCEECCEEFF121AC5CFEDCF021A63
:011BEE00C531
:091C70007BFF7A1B795A021BA9C3
:0E0B33008F418E408D3F8C3E8B428A43894419
:100B4100E4F54EEC4D4E4F7017E94A4B70057F307E
:100B5100020016121B6E8F827583007430020C56D0
:100B6100121B7BEC33502AE5444543454270077F15
:100B71002D120016800D121B6E8F82758300742D4D
:100B8100120985121B79120AC48F418E408D3F8C48
:100B91003E754D017548007547CA75469A75453BC6
:100BA100E4FFFEFDFCAB48AA47A946A845D3120ABB
:100BB100E85003020C41121B79A845120A328F4CEE
:100BC1008E4B8D4A8C49EC4D4E4F7004E54D702390
:100BD100E54C2430FFE544454345427005120016BB
:100BE100800EAE4E121B708E82758300EF12098546
:100BF100E4F54DAF48AE47AD46AC45AB4CAA4BA969
:100C01004AA8491209A7CAEECAC9EDC9C8ECC8C3A6
:100C1100E5419FF541E5409AF540E53F99F53FE50E
:100C21003E98F53EAF48AE47AD46AC45E47B0AFA87
:100C3100F9F8120A328F488E478D468C45020BA176
:100C4100E543454445426010AB42AA43A944854E61
:080C510082758300E41209859D
:010C59002278
:100E57001F2561A8201A5FB421125DC0220D5BCC4B
:100E6700230E59D8241557E4251F55F0262F53FC78
:100E770027425208285B501429764E202A9B4C2C77
:100E87002BC04A382CEE48442E1E46502F55445C42
:100E9700308F426831D1407433173E8034633C8CC5
:100EA70035B13A98370938A4386636B039C734BCF3
:100EB7003B2D32C83C9D30D43E0F2EE03F882CECB2
:100EC70041062AF8428D29044418271045AB251CF2
:100ED7004741232848E121344A861F404C311D4CA5
:100EE7004DE21B584F9C1964515D17705323157CB5
:100EF70054EF138856C4119458A20FA05A830DAC0F
:100F07005C6D0BB85E6009C4605807D0625A05DC97
:100F1700646203E8667301F4688A00006AA1FE0C44
:0C0F27006CB8FC186ECFFA2470E6F830AD
:1016C800F583E493FE740193FFE53425E025E022D9
:1016D800F583C37401939FFFE4939EFEE4228F3544
:1016E8008E348D338C32228F318E308D2F8C2E227A
:0816F8002457F582E4340E22B0
:101B8200C3EF9DEE9C400AD3EF9BEE9A50037F0178
:041B9200227F00228C
:040C5A008E328F3314
:100C5E00E4F5341216D11216F8F583E493FC740100
:100C6E0093FD1216D1245BF582E4340EF583E493E2
:100C7E00FA740193FBAF33AE32121B82EF70030294
:100C8E000D521216D11216F81216C8245BF582E414
:100C9E00340E1216D88F388E37F536F5351216D12A
:100CAE00245DF582E4340E1216C82459F582E4341C
:100CBE000E1216D88F3C8E3BF53AF539AD3AAC395B
:100CCE00120AC48F3C8E3B8D3A8C39AE32AF33E470
:100CDE00FCFDEEC0E0EFC0E01216D11216F8F5835F
:100CEE00E493FE740193FBCAEECAD0E0FFD0E0FE9F
:100CFE00C3EF9BFFEE9AFEED9400FDEC9400FCAB6F
:100D0E003CAA3BA93AA8391209A7AB38AA37A9368B
:100D1E00A8351214CBC8ECC8C9EDC9CAEECACBEFC0
:100D2E00CB1216D12459F582E4340EF583E493FEEA
:100D3E00740193FFE4FCFDEB2FFFEA3EFEED39FD5F
:100D4E00EC38FC220534E534C394365003020C61B2
:050D5E00E4FFFEFDFCB6
:010D6300226D
:01001A0022C3
:10139B001216E6AB35AA34A933A832E8C0E078A719
:1013AB00E6FE08E6FFE4FCFDD0E0F81209A71216F2
:1013BB00E6780E120AF91216E678A9E6FE08E6FFA1
:1013CB00EE3395E0FDFCE5352FF535E5343EF53490
:1013DB00E5333DF533E5323CF532AF35AE34AD3365
:0213EB00FC22E2
:0213ED008D2D44
:1013EF00120C5A1216EF12139B1216EFE52D146002
:1013FF001C14702DE47FE87E03FDFCAB31AA30A9ED
:10140F002FA82E1209A7E47BE87A0B800CAF31AE20
:10141F0030AD2FAC2EE47B03FAF9F81214CB121671
:09142F00EFAF31AE30AD2FAC2E51
:011438002291
:10092D00BB010689828A83E0225002E722BBFE02C8
:09093D00E32289828A83E49322FB
:10094600BB010CE58229F582E5833AF583E0225066
:1009560006E92582F8E622BBFE06E92582F8E222B0
:0D096600E58229F582E5833AF583E49322CA
:10097300BB010689828A83F0225002F722BBFE0163
:02098300F3225D
:10098500F8BB010DE58229F582E5833AF583E8F0A8
:10099500225006E92582C8F622BBFE05E92582C854
:0209A500F2223C
:1009A700E88FF0A4CC8BF0A42CFCE98EF0A42CFCEF
:1009B7008AF0EDA42CFCEA8EF0A4CDA8F08BF0A46D
:1009C7002DCC3825F0FDE98FF0A42CCD35F0FCEBCC
:1009D7008EF0A4FEA9F0EB8FF0A4CFC5F02ECD3991
:0F09E700FEE43CFCEAA42DCE35F0FDE43CFC22FE
:1009F60075F008758200EF2FFFEE33FECD33CDCCB8
:100A060033CCC58233C5829BED9AEC99E58298403A
:100A16000CF582EE9BFEED9AFDEC99FC0FD5F0D617
:100A2600E4CEFBE4CDFAE4CCF9A88222B800C1B941
:100A36000059BA002DEC8BF084CFCECDFCE5F0CB7F
:100A4600F97818EF2FFFEE33FEED33FDEC33FCEBB8
:100A560033FB10D703994004EB99FB0FD8E5E4F973
:100A6600FA227818EF2FFFEE33FEED33FDEC33FC60
:100A7600C933C910D7059BE99A4007EC9BFCE99A54
:100A8600F90FD8E0E4C9FAE4CCFB2275F010EF2F99
:100A9600FFEE33FEED33FDCC33CCC833C810D70799
:100AA6009BEC9AE899400AED9BFDEC9AFCE899F8D4
:0E0AB6000FD5F0DAE4CDFBE4CCFAE4C8F92267
:1014CB00C2D5E830E70FB2D5E4C39BFBE49AFAE44C
:1014DB0099F9E498F8EC30E717B2D5121501120A16
:1014EB0032E4C39BFBE49AFAE499F9E498F880039D
:1014FB00120A3230D50DE4C39FFFE49EFEE49DFD3E
:04150B00E49CFC223E
:0E0AC400C3E49FFFE49EFEE49DFDE49CFC2243
:100AD200EB9FF5F0EA9E42F0E99D42F0EC6480C89B
:060AE20064809845F0223B
:100AE800EB9FF5F0EA9E42F0E99D42F0E89C45F064
:010AF80022DB
:100AF900E86010ECA2E713FCED13FDEE13FEEF1313
:040B0900FFD8F022FF
:100B0D00D083D082F8E4937012740193700DA3A377
:100B1D0093F8740193F5828883E47374029368608B
:060B2D00EFA3A3A380DF8B
:00000001FF
